:100000000C946A000C9400000C9400000C94000006
:100010000C9400000C9400000C9400000C94000060
:100020000C9400000C9400000C9400000C94000050
:100030000C9400000C9400000C9400000C94000040
:100040000C94CC000C9400000C9499000C940000CB
:100050000C9400000C9400000C9400000C94000020
:100060000C9400000C9400001027E80364000A00C0
:1000700001000010000110000100000000000A0053
:100080000000000000000000000000000000000070
:100090000000000000000000000000000000000060
:1000A0000000000000000000000000000000000A46
:1000B0000A0A0A0A0A0A0A0A0A0A0A0A0A0A0A00AA
:1000C000020002007A00020004007C000100090323
:1000D0007E000000F894EE27EFBBF1E0F5BFE5BF2E
:1000E0008DE0A2E0BB27ED938A95E9F780E098E0E8
:1000F000A0E0B1E0ED930197E9F7E0ECF0E0859145
:100100009591009761F0A591B59105901590BF016B
:10011000F00105900D920197E1F7FB01F0CFE8E0C7
:10012000EEBBEFEFEDBFE8E0EEBFC0E0D3E00C9434
:100130004F03AA93EA93FA93EFB7EA931A930A93B9
:100140001091C0000091C600E12FEC71E9F4E0913C
:10015000E203EF5FE093E203E150F0E0E753FC4F8E
:100160000083A091E203A93119F4E0E0E093E203F7
:10017000A091E403AF5FA093E403A93129F4E0E088
:10018000E093E403689435F809911991E991EFBF80
:10019000F991E991A99118950A921A926A937A9322
:1001A0008A939A93AA93BA93EA93FA93EFB7EA934E
:1001B000E0913903F0913A033196E0933903F093DB
:1001C0003A030E949C1DE1E5F1E00E94AA270E2E51
:1001D0000E949C1DE3EAF2E00E94AA27E02909F4AC
:1001E000C4C1A0913703B0913803E4E1F0E00E946C
:1001F000BC270E2EE0910603F0E074970E94B02712
:100200000E22A0911E03EEE00E94A027E02121F023
:10021000E0911E03EF5F03C025FC03C0E0E0E09324
:100220001E03A0911E03AE3011F4689425F8E091EE
:100230003703E0930603A0912703A13029F4F79B2D
:1002400002C0F79801C0F79AE1E02E260E94A11D96
:100250000E94AA1DE093B103F093B2036093B3032D
:100260007093B4030E94B11DA5E9B3E00E94B61DCE
:100270000E94BD1DA1ECB3E00E94B61D0E94C21DEC
:100280000E94CB1D0E94D626E0939503F09396031F
:100290006093970370939803A091C103B091C20338
:1002A0008091C3039091C403E0E0F0E060E772E462
:1002B0000E94D626E093C103F093C2036093C30368
:1002C0007093C4030E94D01D0E94D51D0E2E0E9463
:1002D000DA1D0E94D51DE02161F1E091C103F0918A
:1002E000C2036091C3037091C4030E94C21D0E94A7
:1002F000D626E093BD03F093BE036093BF037093D3
:10030000C0030E94DF1DABE4B3E00E94E81DA09192
:10031000BD03B091BE038091BF039091C0030E94C2
:10032000AA1DE0939D03F0939E0360939F03709337
:10033000A0030E94ED1DE0E0F0E06AE774E40E9493
:10034000F61D0E94FB1D0E943826E093A503F09342
:10035000A6036093A7037093A8030E94041E0E9443
:100360000D1E0E94201EA1E8B3E00E94C7250E9436
:100370009E280E94251E0E94ED1D0E94FE250E94BF
:10038000F61DE093B503F093B6036093B703709343
:10039000B8030E942E1E0E9438260E94371E0E941B
:1003A000041EA5E2B0E080E090E00E94401EA9E6B5
:1003B000B3E00E944F1E0E94A11D0E94F4283CF54C
:1003C000A091B503B091B6038091B7039091B803A3
:1003D0000E94541E7F936F93FF93EF93A091B103FC
:1003E000B091B2038091B3039091B4030E94541E64
:1003F000AF91BF918F919F910E94D626E093AD035C
:10040000F093AE036093AF037093B00309C0E0E0D4
:10041000E093AD03E093AE03E093AF03E093B0034A
:100420000E945B1EACE2B3E00E94C525EC930E94E3
:10043000641E0E946D1E0E9438260E94761EE09166
:100440009503F091960360919703709198030E9431
:100450007F1E0E941B2768F5E0919D03F0919E038B
:1004600060919F037091A0030E947F1E0E94382616
:10047000E0939903F0939A0360939B0370939C031A
:100480000E947F1E0E94881E0E943126DF01CB0140
:100490000E94DF1D0E94D626A0E0B0E081E695E430
:1004A0000E948826A5E6B3E00E944F1E689424F8B7
:1004B00002C0E0E12E260E94641E0E94911E0E944E
:1004C0003826E093A103F093A2036093A3037093F3
:1004D000A4030E94911EE0E0F0E060E87FE30E9448
:1004E0001B2709F008F416C0E093A103E093A203D0
:1004F000E093A303E093A4030E949A1EEF5FFF4FD3
:100500006F4F7F4F0E94A31E0E949A1EA8E3B0E087
:100510000E94C9280E94AC1EA034E2E4BE07EFE0AE
:100520008E07E0E09E0778F0E0E0E0935703E09369
:100530005803E0935903E0935A03A8E3B0E00E9404
:10054000B51E0E94C9280E946D1E0E94BA1EABE310
:10055000B3E00E94E81DA0911C03AC3308F4F298AC
:10056000A0911C03AC3309F4F29A0E949C1DA33A9B
:10057000E2E0BE0709F06AC0A0911B030E94BE1E04
:100580000E94C31E0E94B51E0E94C2270E94CC1E5C
:10059000E02191F0E0911C03EF5FE0931C03E091F8
:1005A0001B03F0E03296A0911C03B0E0EA17FB07B2
:1005B00019F4ECE3E0931C03E0E0E0933903E093EB
:1005C0003A03C3940E94D31EE8E5F2E00E94B627E6
:1005D0000E2E0E94D81EE021E9F0E0914F03F09129
:1005E00050033196E0934F03F09350030E94D31EC3
:1005F0000E94DD1EEA1BFB0BE0935503F0935603AC
:100600000E94C31E0E94F4282CF4E0E0E0934F0304
:10061000E0935003ECE3EC15C9F4CC24E091000323
:10062000EF5FE0930003A0910003AC3379F4E0E0C6
:10063000E0930003E0910103EF5FE0930103A091D9
:100640000103A43119F4E0E0E0930103E991EFBF65
:10065000F991E991B991A9919991899179916991CA
:10066000199009901895AA93E881E066E0937C00C0
:1006700085E28A95F1F7E0917A00E064E0937A00F0
:10068000E0917A00E071E1F3E0917A00E061E093BB
:100690007A00E0917800F091790021960895EF9723
:1006A00022978FE3A2E0B0E0E0E8F0E00E940929A1
:1006B000FF2401E021E0E0E8E0936100E0E0E09366
:1006C0006100EFE0E4B9E1E0E5B9E0E0E7B9E4E0DA
:1006D000E8B9EAEFEAB9E7E6EBB9E0E0E4BDE3E068
:1006E000E5BDE0E0E6BDE7BDE8BDE1EAE0938000FE
:1006F000E2E0E0938100E0E0E0938500E093840095
:10070000E0938700E0938600E0938900E0938800FF
:10071000E0938B00E0938A00E093B600E1EAE09377
:10072000B000E2E0E093B100E0E0E093B200E093DB
:10073000B300E093B400E1E0E0936E00E0E0E0930A
:100740006F00E0937000E0936900EDBBE0936800F8
:10075000E093C000E8E9E093C100E6E0E093C20066
:10076000E0E0E093C500E7E4E093C400E0E8E0BF28
:10077000E0E0E0937F00E0937E00E0E6E0937C0021
:10078000E7E2E0937A00E0E0E0937B00ECBDE093E9
:10079000BC007894A2E3B0E00E948E255F9A0E948C
:1007A000E21E0E94F21E0E94FF1EEAE09E1620F446
:1007B000A8E2B0E00E94091FEAE08E1650F4AEE213
:1007C000B0E00E94091FA6E3B0E00E94091F6894F0
:1007D00026F8EAE0AE1618F4689430F827F8689422
:1007E00033F80E940E1F0E94151F0E941C1FE8EC88
:1007F000F0E0E0935F03F0936003E2E1E093100325
:10080000A0E0B0E00E94BD28E0931103A1E0B0E0B9
:100810000E94BD28E0931203A2E0B0E00E94BD2830
:10082000E0931303A3E0B0E00E94BD28E09315031A
:10083000A4E0B0E00E94BD28EF8BA5E0B0E00E94EC
:10084000BD28E88FA6E0B0E00E94BD28E98FA7E0B0
:10085000B0E00E94BD28E0931603A8E0B0E00E943B
:10086000BD28E0931703A9E0B0E00E94BD28E09303
:100870001803F798F198AAE0B0E00E94BD28E09331
:100880001B03A6E2B0E00E94B9280E94231FA4E146
:10089000B0E00E94BD28EB8BA5E1B0E00E94BD282E
:1008A000EC8BA6E1B0E00E94BD28ED8BABE0B0E0A0
:1008B0000E94BD28EF87ACE0B0E00E94BD28E88B25
:1008C000ADE0B0E00E94BD28E98BAAE2B0E00E9452
:1008D000B928ED83FE83AEE0B0E00E94BD28E0932E
:1008E0002803AFE0B0E00E94BD28E0932A03A0E116
:1008F000B0E00E94BD28E0932903A8E3B0E00E9485
:10090000B5280E94A31EA8E2B0E00E94B928A1E980
:10091000B3E00E94281F0E94881EABE3B3E00E9450
:10092000E81D0E946D1E0E94CB1D0E94D6260E94CB
:10093000761EA1E1B0E00E94BD283E2FACE2B0E0FF
:100940000E94B928E987FA87A2E1B0E00E94BD2899
:10095000EB8FA3E1B0E00E94BD28EA8FAEE2B0E0E9
:100960000E94B928A5EAB3E00E94281FA6E3B0E0E0
:100970000E94B928A5ECB3E00E94281F0E942E1EF9
:100980000E94CB1D0E94D6260E94371EA0E3B0E035
:100990000E94B9280E942F1FA4E3B0E00E94B9284A
:1009A0000E947D270E94341FA7E1B0E00E94BD286D
:1009B0000E94042923F8A2E3B0E00E94B9280E9413
:1009C0003D1FA8E1B0E00E94BD28E0930803A9E123
:1009D000B0E00E94BD28E0930A03AAE1B0E00E94C3
:1009E000BD28E0930B03ABE1B0E00E94BD28E0938B
:1009F0000C03ACE1B0E00E94BD28E0930D03ADE133
:100A0000B0E00E94BD28E0930E03AEE1B0E00E948A
:100A1000BD28E0931F03AFE1B0E00E94BD28E09342
:100A20002003A0E2B0E00E94BD28E0932103A1E2F0
:100A3000B0E00E94BD28E0932203A2E2B0E00E9451
:100A4000BD28E0932303A3E2B0E00E94BD28E09319
:100A50002403A4E2B0E00E94BD28E0932503A5E2B0
:100A6000B0E00E94BD28E0932603A0910303A431C7
:100A700028F4E0910303EF5FE0930303A0910303E5
:100A8000A431A1F4E0E0E0932E03E0932F03EBE028
:100A9000F0E0E0935303F0935403E8EBE09330036A
:100AA000E0E0E093E203EAE0E0930303A091E203D5
:100AB000AB30C1F4E091CC03E0932E03E091CD0381
:100AC000E0932F03E091CE03F0E0E0935303F09323
:100AD0005403E091CF03E0933003E0E0E093E203BE
:100AE000E0930303A091E203AC30C0F0E0E0E093B8
:100AF000C903E093CA03E093CB03E093CC03E093F4
:100B0000CD030E940E1FE0E0E093D003E093D103F9
:100B1000E093D203E093D303E093E203E8EC5E16A4
:100B200030F45394E4E1E51511F4E1E04E2EA4E134
:100B3000B0E00E948E250E94421F3B9798F1A0E0F2
:100B40000E944B1F662777270E94521F0E94251E76
:100B5000A8EEB3E080E090E00E940D28DF01CB0119
:100B60000E945B1F662777270E944F280E94521F12
:100B7000E0910903EF5FE0930903E0910803A0917E
:100B80000903AE1768F00E94251EE0937D03F093E1
:100B90007E0360937F0370938003E0E0E09309039A
:100BA000E894F3F8E7E2E0937A000E94E21EA2E004
:100BB0000E944B1FDF01E5E0F0E00E941228BE2EEC
:100BC0000E94601F0E94F21E0E94671F0E94601F09
:100BD000A5E00E94711F1E2FE7E2E0937A000E94B9
:100BE000421FDE2E0E94601F0E94FF1EE7EAE09374
:100BF0007A00A6E00E94711FED87E7E2E0937A0099
:100C0000E1E0E51591F50E94761FE2E3F0E00E9435
:100C1000BC270E2E0E947B1F0E94B627E02111F0F8
:100C2000E5E0EC87A12FE2E30E94A5270E2EEAEF74
:100C30000E94A027E02111F0E6E0EC870E947B1FD4
:100C40000E94BC270E2E0E947F1FE02911F0E7E0D2
:100C5000EC87A12FEAEF0E94A5270E2EEEE10E945D
:100C6000A027E02911F0E8E0EC870E947B1F0E949A
:100C7000BC270E94851F39F0E1E0EC87E8E2F0E054
:100C80000E94911F07C00E947F1F0E94851F11F0C4
:100C9000E2E0EC87A12FEAEF0E94A5270E94851FC2
:100CA00011F0E3E008C0A12FEEE10E94A0270E940E
:100CB000851F19F0E4E0EC871CE3AC850E94961FC9
:100CC000AC85E7E00E9487270E2AE1E00E94872793
:100CD0000E2AE2E00E948727E02929F0E12FF0E0C8
:100CE0000E94911F18E2AC850E949B1FAC85E8E032
:100CF0000E948727E02909F018E20E94A01F0E94A5
:100D0000A61F0E94A027E021D1F06894F3F80130DB
:100D100021F4F398F49A02E012C0023059F4F498E6
:100D2000F59AA98DA13010F003E003C0F598F39A6D
:100D300001E005C0033019F4F598F39A01E00E9430
:100D4000761FD39708F457C00E94B01F0E94B51FAA
:100D5000E02F0E94BC1F20F0E8ECF0E00E94911F01
:100D6000E02F0E94CC1F0E94DC1FAC91A13008F440
:100D700041C00E94E31F0E94EC1F0E94FF284CF418
:100D80000E94DC1F0E94F81F0E9447270E94032038
:100D900023C00E940C200E940E20EF930E940C2082
:100DA0000E941720AF91EA2379F00E94DC1F0E9475
:100DB000F81F0E944C27A0936D03B0936E0380939D
:100DC0006F039093700308C00E940C200E942020A3
:100DD0001CF00E942A200EC0A0916D03B0916E03FA
:100DE00080916F03909170030E9439200E944F28D8
:100DF0000E94911F04C00E943E200E942A200E944F
:100E000044200E944A200E220E944F20E02139F007
:100E1000E0913503E0931D036894F0F821F80E94F7
:100E2000B01F309721F4E0E0E0931E0306C0A091CC
:100E30001E03A23010F4E89425F80E94B01FE0933E
:100E40003703F09338030E94B01F309719F4E894E9
:100E500021F815C0A0E021FCA1E0E0E00E94872776
:100E60000E2EA0911D03E0E00E94A527E02139F09D
:100E7000E0E0E0931D030E943E20E89422F8E09118
:100E800005030E94761FF0E0AE17BF0720F0E09147
:100E90003503E0930503E0910503F0E035970E94E8
:100EA000761FAE17BF0770F4E0913503E09305039A
:100EB00025FE08C0E2E0E0932B03E89425F8E0E08B
:100EC000E0931E03A0911D03A13080F0689422F8E6
:100ED0000E94B01FA0911D03B0E0AE17BF0728F01D
:100EE000E0911D03F0E00E94911F02C0E89422F8F7
:100EF0000E9456200E9459200E94D2270E22A091C3
:100F000028030E9460201E2E0E9456200E94592015
:100F10000E94CA270E22A09129030E9460201E2A47
:100F20000E945620A12FE2E30E94A527E021E1299B
:100F300079F00E943E20A0912B03A13021F4EAE039
:100F4000F0E00E94911FE0912B03E150E0932B030E
:100F50000E9465200E22A0E031FCA1E00E946020EA
:100F600031F0689431F80E94B01F0E947B200E94EB
:100F70006520E02161F10E9480200E948820A4F079
:100F8000A0917903B0917A03ED81FE81EA1BFB0BFE
:100F9000A3E0B0E00E9408280E949020AE1BBF0B87
:100FA000A0936103B09362030E9480200E94F42802
:100FB0002CF40E94952032970E947B20A09162031E
:100FC000AA232AF4E0E0E0936103E09362030E9425
:100FD0009A200E94FA2874F50E949A200E944C27B9
:100FE0000E94882074F0AD81BE81E0917903F09178
:100FF0007A03EA1BFB0B0E949020EA0FFB1F0E9462
:101000007B200E949A200E944C27A230E0E0BE077D
:10101000E0E08E07E0E09E072CF00E9495203196DC
:101020000E947B200E949020A93CE0E0BE0714F0C3
:101030000E94151F0E9495200E94761FAE17BF07C1
:1010400010F4E89431F80E9495200E94761FEA1768
:10105000FB0720F40E9495200E94911F0E94A72068
:101060000E9441270E2EA0E032FCA1E00E946020E9
:1010700041F0689432F80E94B620E0936303F09345
:1010800064030E94A7200E941B2709F008F435C0C2
:101090000E94BB20DF01CB01E0E0F0E060E070E403
:1010A0000E941B2709F008F410C00E94BB20DF013A
:1010B000CB01E985FA850E94CA200E94D1200E94B6
:1010C000D620A3E6B3E00E944F1E0E94BB200E94E0
:1010D000EA2854F4EB8DF0E00E94D120AE1BBF0B48
:1010E000A0936303B0936403A0916403AA232AF43A
:1010F000E0E0E0936303E09364030E94A7200E9472
:101100001B27D0F50E94DB20DF01CB01E0E0F0E0FF
:1011100060E470E40E941B2709F008F416C00E94E6
:10112000DB20A0E0B0E080EA90E40E948826DF01A6
:10113000CB010E94E6200E947D270E94FE250E948E
:101140003826A3E6B3E00E944F1E0E94DB200E94D7
:10115000EA2854F4EA8DF0E00E94D120EA0FFB1F48
:10116000E0936303F09364030E94D120A13DE7E084
:10117000BE0714F00E941C1F0E94B620DF010E94CF
:10118000E620AE17BF0710F4E89432F80E94B620AC
:10119000DF010E94E620EA17FB0720F40E94D1201D
:1011A0000E94EB200E94F0200E94D2270E2EA0E089
:1011B00034FCA1E00E94602031F0689434F80E9471
:1011C000B6200E94F7200E94F0200E94FA285CF5C9
:1011D0000E94FC200E9488209CF0E0911203F0E025
:1011E000A0917503B0917603AE1BBF0BE3E0F0E076
:1011F0000E940521AE1BBF0BA0936B03B0936C0341
:101200000E94FC200E94F4282CF40E940C213297AA
:101210000E94F720A0916C03AA232AF4E0E0E09357
:101220006B03E0936C030E94F0200E94FF288CF572
:101230000E941121A430E0E0BE07E0E08E07E0E06C
:101240009E078CF0A0911203BB27E0917503F091EB
:101250007603AE1BBF0BE2E0F0E00E940521EA0F2F
:10126000FB1F0E94F7200E9411210E94F4282CF4F9
:101270000E940C2132960E94F720A0916B03B0913E
:101280006C03A13DE7E0BE0724F0E0EDF7E00E942B
:10129000F7200E94B620DF010E940C21AE17BF0785
:1012A00010F4E89434F80E94B620DF010E940C216B
:1012B000EA17FB0730F4A0916B03B0916C030E9416
:1012C000EB201333D8F0A0911D03A13018F0E2E019
:1012D000E0932B03E0E0E0931D03E12FF0E0F297B1
:1012E0000E947D270E94FE25A6EFB8E28CE99FE3CD
:1012F0000E9488260E94C5251E2F01C010E00E9472
:10130000B01FEB83FC83AB2DE4E60E94A0270E2EDA
:10131000A0E0F099A1E0E1E00E9487270E94CC1EA6
:101320000E22AA81EDE50E948C27E0211E2E0E944C
:10133000DD1E0E94D31E0E94AA270E9421210E9426
:10134000D81EE021E12909F46AC0E0913B03F09145
:101350003C03A8E2B0E00E94D1280E9429210E940B
:101360007B210E9481210E9486210E948B21EC8991
:10137000A5E1B0E00E947B21ED89A6E1B0E00E94EA
:101380007B21EF85ABE0B0E00E947B21E889ACE0F7
:10139000B0E00E947B21E989ADE0B0E00E947B21B2
:1013A0000E9498210E94A7210E94AC21E32FA1E175
:1013B000B0E00E947B210E94B121EA8DA3E1B0E060
:1013C0000E947B210E94BF210E94EF210E94FD21EB
:1013D0000E9402220E9407220E940C220E941122D7
:1013E0000E942E1E0E94BA1E0E9416220E942522D2
:1013F0000E942A220E942F220E9434220E94392217
:101400000E943E220E944322A4E6B0E00E948E2564
:101410005F98A8EEB3E00E948E255F98FECFAA2DBC
:101420000E944A220E944A20E02131F0E894F2F81A
:1014300027F8E0E0E09334030E944F220E944A2004
:10144000E02171F0E0913403EF5FE0933403A09169
:101450003403AA3029F4E0E0E0933403E093270357
:101460000E944F220E945C220E944A20E02171F0DB
:101470006894F2F8E0912703EF5FE0932703A091CF
:101480002703A33019F4E1E0E0932703E091270359
:10149000E03029F4E0E0E093B400F7980FC0A091A9
:1014A0002703A13019F4E091180306C0A091270387
:1014B000A23021F4F79AEFEFE093B4000E94761F78
:1014C0000E94D51D0E2EA12FE0E00E94A5270E221E
:1014D000A0E022FCA1E00E94602001F1E091040361
:1014E000EF5FE0930403A0910403E5E00E94A527C9
:1014F0000E2EE4E10E94A027E02141F0E0910403D8
:10150000E170AFEFEA02F001E093B400A0910403B0
:10151000A03118F0E0E0E093040326C0A0E030FC26
:10152000A1E0E1E00E9487270E2EA09127030E94F0
:101530006020D1F0E0913303EF5FE0933303A0919B
:101540003303A13019F4EFEFE093B400A09133031B
:10155000A33019F4E0E0E093B400A0913303A43089
:1015600019F4E0E0E0933303E0911703E093B30054
:10157000EAE0E81518F4E894F1F826F80E946422ED
:10158000A0E026FCA1E00E946A22A0E0F1FCA1E01C
:101590000E946A220E944A20E02139F16894F1F801
:1015A000E0910F03EF5FE0930F03E0E0EB87AB8583
:1015B000A53088F40E946F22A081A13018F0E5E0E8
:1015C000EB8705C0E0910F03EF5FE0930F03EB851E
:1015D000EF5FEB87ECCFA0910F03A53018F0E0E0B0
:1015E000E0930F030E946F2220810E946422A09149
:1015F0001A03EFEF0E94A027E02121F0E0911A03E7
:10160000EF5F03C0E894F1F8E0E0E0931A03A091E3
:101610001A03A43109F06DC0AA81E0E00E949B2763
:101620000E2E0E944A20E02119F0EA81E150EA835F
:10163000233610F423E65DC021E0E0E0E0930F03E1
:101640000E9429210E947B210E9481210E948621E3
:101650000E948B21EC89A5E1B0E00E947B21ED89FD
:10166000A6E1B0E00E947B21EF85ABE0B0E00E94F4
:101670007B21E889ACE0B0E00E947B21E989ADE004
:10168000B0E00E947B210E9498210E94A7210E9425
:10169000AC21E32FA1E1B0E00E947B210E94B121A7
:1016A000EA8DA3E1B0E00E947B210E94BF210E944D
:1016B000EF210E94FD210E9402220E9407220E9427
:1016C0000C220E9411220E942E1E0E94BA1E0E940D
:1016D00016220E9425220E942A220E942F220E9466
:1016E00034220E9439220E943E220E944322E1E0DD
:1016F0004E2E0E946422A0E0F1FCA1E00E946A222A
:10170000AA81E4E60E9496270E94752251F068940F
:10171000F1F8EA81EF5FEA83AA81A43611F4E0E0F0
:10172000EA83EAE0E91510F4E894F0F80E94442016
:101730000E944F200E22AA81E0E00E9491270E9481
:10174000752251F06894F0F8EA81E150EA83AA81A9
:10175000AF3F11F4E3E6EA830E94A01F0E947C22BF
:10176000C1F00E948222A9F4A0913103A43119F49E
:10177000E7E0E0933103E0E0E0933203E894F3F82C
:10178000A0913103A33028F0E0913103E150E093C0
:101790003103AA2DEAE00E94A0270E2E0E947C228F
:1017A000C1F00E948222A9F4A0913103A43119F45E
:1017B000E7E0E0933103E0E0E0933203E894F2F8ED
:1017C000A0913103A33028F0E0913103E150E09380
:1017D0003103AA2D0E944A22AD2DEAE00E94A527DE
:1017E000E02131F0E0E0E0933203E4E1E093310303
:1017F000EAE0ED1510F4E894F3F80E94A01F0E94AF
:10180000A61F0E948727E02109F438C26894F3F8E4
:10181000AA81A13049F4A0911103A13028F4E091EC
:101820001103EF5FE0931103AA81A23049F4A09164
:101830001203A23328F4E0911203EB5FE09312034A
:10184000AA81A33049F4A0911303A43628F4E091AF
:101850001303EF5FE0931303AA81A43049F4A0912E
:101860001503A83228F4E0911503EF5FE093150308
:10187000AA81A53031F4AF89A43618F4EF89EF5F5F
:10188000EF8BAA81A63031F4A88DA43618F4E88D28
:10189000EF5FE88FAA81A73031F4A98DA43618F440
:1018A000E98DEF5FE98FAA81A83049F4A091160372
:1018B000AF3F28F4E0911603EF5FE0931603AA818F
:1018C000AD3069F4A0913D03B0913E03A433E8E04C
:1018D000BE0728F40E945B1F31960E94231FAA8135
:1018E000AE3031F4AB89A43618F4EB89EB5FEB8BA7
:1018F000AA81AF3031F4AC89A43618F4EC89EB5FDF
:10190000EC8BAA81A03131F4AD89A43618F4ED89AD
:10191000EB5FED8BAA81A13131F4AF85A83C18F4BF
:10192000EF85EB5FEF87AA81A23131F4A889A83C4B
:1019300018F4E889EB5FE88BAA81A33131F4A98917
:10194000A83C18F4E989EB5FE98BAA81A43169F41A
:10195000A0914D03B0914E03A835E2E0BE0728F4F4
:101960000E94DD1E7E960E943D1FAA81A53159F47A
:10197000AD81BE81A33AE1E0BE0728F4ED81FE818E
:101980003196ED83FE83AA81A63149F4A091280304
:10199000A13028F4E0912803EF5FE0932803AA81A7
:1019A000A73149F4A0912A03A23328F4E0912A0335
:1019B000EF5FE0932A03AA81A83149F4A09129039B
:1019C000A13028F4E0912903EF5FE0932903AA8175
:1019D000A93119F43F3008F43F5FAA81AA3159F4C4
:1019E0000E948D22AC3BE2E0BE0728F40E949222C6
:1019F00031960E942F1FAA81AB3191F40E94972249
:101A0000A73EE3E0BE07E0E08E07E0E09E0740F47B
:101A10000E94041EEF5FFF4F6F4F7F4F0E94341FE5
:101A2000AA81AC3161F4A0E023FCA1E0A13038F43C
:101A3000E0E023FCE1E0EF5F0E94042923F8AA81A3
:101A4000AD3169F40E94D01DAE3DE3E0BE0738F42D
:101A50000E94B11D3A96E0934503F0934603AA8194
:101A6000AE3169F40E94DA1DA835E2E0BE0738F411
:101A70000E94BD1D3A96E0935103F0935203AA8150
:101A8000AF3149F4A0910803AA3028F4E09108038B
:101A9000EF5FE0930803AA81A03249F4A0910A0302
:101AA000AA3028F4E0910A03EF5FE0930A03AA81C9
:101AB000A13249F4A0910B03AA3028F4E0910B0362
:101AC000EF5FE0930B03AA81A23249F4A0910C03CB
:101AD000AA3028F4E0910C03EF5FE0930C03AA8195
:101AE000A33249F4A0910D03AA3028F4E0910D032C
:101AF000EF5FE0930D03AA81A43249F4A0910E0395
:101B0000AA3028F4E0910E03EF5FE0930E03AA8160
:101B1000A53249F4A0911F03A13028F4E0911F03DE
:101B2000EF5FE0931F03AA81A63249F4A09120033E
:101B3000A13028F4E0912003EF5FE0932003AA8115
:101B4000A73249F4A0912103A13028F4E0912103A8
:101B5000EF5FE0932103AA81A83249F4A091220308
:101B6000A13028F4E0912203EF5FE0932203AA81E1
:101B7000A93249F4A0912303A13028F4E091230372
:101B8000EF5FE0932303AA81AA3249F4A0912403D2
:101B9000A23028F4E0912403EF5FE0932403AA81AC
:101BA000AB3249F4A0912503A13028F4E09125033C
:101BB000EF5FE0932503AA81AC3249F4A09126039C
:101BC000A13028F4E0912603EF5FE0932603AA8179
:101BD000AC3549F4A0910703AA3F28F4E09107032C
:101BE000E65FE0930703AA81AD3531F4AC8DA730F1
:101BF00018F4EC8DEF5FEC8FAA81AE3549F4A9851E
:101C0000BA851A9728F4E985FA853196E987FA8723
:101C1000AA81AF3531F4AB8DAA3018F4EB8DEF5FAC
:101C2000EB8FAA81A03631F4AA8DAA3018F4EA8D80
:101C3000EF5FEA8FAA81A13649F4A0911B03AC3370
:101C400028F4E0911B03EF5FE0931B03AA81A23607
:101C500049F4A0911803AA3F28F4E0911803E65F25
:101C6000E0931803AA81A33649F4A0911703AA3F71
:101C700028F4E0911703E65FE0931703EAE0EA1522
:101C800010F4E894F2F8AA2DEAE00E94A0270E2EA4
:101C90000E945C220E947C2209F437C26894F2F808
:101CA000AA81A13049F4A0911103A13028F0E0915C
:101CB0001103E150E0931103AA81A23049F4A091ED
:101CC0001203AB3028F0E0911203E550E0931203C9
:101CD000AA81A33049F4A0911303AD3328F0E09119
:101CE0001303E150E0931303AA81A43049F4A091B7
:101CF0001503A53128F0E0911503E150E093150399
:101D0000AA81A53031F4AF89A13018F0EF89E150F4
:101D1000EF8BAA81A63031F4A88DA13018F0E88DA0
:101D2000E150E88FAA81A73031F4A98DA13018F0D5
:101D3000E98DE150E98FAA81A83049F4A0911603FA
:101D4000A13028F0E0911603E150E0931603AA8138
:101D5000AD3069F4A0913D03B0913E03AD36E7E0AC
:101D6000BE0728F00E945B1F31970E94231FAA81A3
:101D7000AE3031F4AB89A63018F0EB89E550EB8B2F
:101D8000AA81AF3031F4AC89A63018F0EC89E55067
:101D9000EC8BAA81A03131F4AD89A63018F0ED8921
:101DA000E550ED8BAA81A13131F4AF85A13018F057
:101DB000EF85E550EF87AA81A23131F4A889A130DF
:101DC00018F0E889E550E88BAA81A33131F4A9899C
:101DD000A13018F0E989E550E98BAA81A43161F4BA
:101DE000A0914D03B0914E030E94F02828F40E9468
:101DF000DD1E7E970E943D1FAA81A53159F4AD8159
:101E0000BE81A332E1E0BE0728F0ED81FE8131976B
:101E1000ED83FE83AA81A63149F4A0912803A13065
:101E200028F0E0912803E150E0932803AA81A7312C
:101E300049F4A0912A03A23028F0E0912A03E1504E
:101E4000E0932A03AA81A83149F4A0912903A13083
:101E500028F0E0912903E150E0932903AA81A931F8
:101E600019F4323008F03150AA81AA3159F40E9495
:101E70008D22A935E2E0BE0728F00E949222319718
:101E80000E942F1FAA81AB3191F40E949722AB30A0
:101E9000E0E0BE07E0E08E07E0E09E0740F00E9431
:101EA000041EE150F040604070400E94341FAA813F
:101EB000AC3179F4A0E023FCA1E0A13050F0A0E027
:101EC00023FCA1E0E1E00E94B128EA1B0E94042962
:101ED00023F8AA81AD3161F40E94D01D0E94F02840
:101EE00038F40E94B11D3197E0934503F093460307
:101EF000AA81AE3161F40E94DA1D0E94F02838F404
:101F00000E94BD1D3197E0935103F0935203AA81C3
:101F1000AF3149F4A0910803A23028F0E091080302
:101F2000E150E0930803AA81A03249F4A0910A038A
:101F3000A23028F0E0910A03E150E0930A03AA815D
:101F4000A13249F4A0910B03A13028F0E0910B03DA
:101F5000E150E0930B03AA81A23249F4A0910C0353
:101F6000A13028F0E0910C03E150E0930C03AA812A
:101F7000A33249F4A0910D03A13028F0E0910D03A4
:101F8000E150E0930D03AA81A43249F4A0910E031D
:101F9000A13028F0E0910E03E150E0930E03AA81F6
:101FA000A53249F4A0911F03A13028F0E0911F034E
:101FB000E150E0931F03AA81A63249F4A0912003C7
:101FC000A13028F0E0912003E150E0932003AA81A2
:101FD000A73249F4A0912103A13028F0E091210318
:101FE000E150E0932103AA81A83249F4A091220391
:101FF000A13028F0E0912203E150E0932203AA816E
:10200000A93249F4A0912303A13028F0E0912303E1
:10201000E150E0932303AA81AA3249F4A09124035A
:10202000A13028F0E0912403E150E0932403AA8139
:10203000AB3249F4A0912503A13028F0E0912503AB
:10204000E150E0932503AA81AC3249F4A091260324
:10205000A13028F0E0912603E150E0932603AA8105
:10206000AC3539F4A0910703A13018F0E0E0E0931B
:102070000703AA81AD3531F4AC8DA13018F0EC8D99
:10208000E150EC8FAA81AE3551F4A985BA850E9442
:10209000F02828F4E985FA853197E987FA87AA813B
:1020A000AF3531F4AB8DA13018F0EB8DE150EB8FF3
:1020B000AA81A03631F4AA8DA13018F0EA8DE15042
:1020C000EA8FAA81A13649F4A0911B03A13028F020
:1020D000E0911B03E150E0931B03AA81A23649F46F
:1020E000A0911803AB3028F0E0911803EA50E09378
:1020F0001803AA81A33649F4A0911703A13028F050
:10210000E0911703EA50E093170323FC26C0E09107
:102110002F03A9EBB3E0FF27662777270E94FE2550
:102120000E949E28A091B903B091BA038091BB038D
:102130009091BC030E94F4283CF40E94A0220E94CB
:10214000A9220E94B02209C0E0E0E093A903E09335
:10215000AA03E093AB03E093AC0323FE0BC0AD8571
:102160000E94B922A9EBB3E00E94281F0E94A0227E
:102170000E94B0220E94A022ADE2B3E00E94C525D9
:10218000EC93F0915303E0E0DF01E0913003F0E0E5
:10219000EA0FFB1FA9E8B3E00E94B61D0E94BF2210
:1021A000A0E0B0E080E192E40E94D6267F936F9396
:1021B000FF93EF930E948D220E94C822AF91BF919E
:1021C0008F919F910E94CA20E0938903F0938A0324
:1021D00060938B0370938C030E94CD22E0E0F0E0CB
:1021E00060E87FE30E9441270E2E0E94CD22E0E0AE
:1021F000F0E068E472E40E943B27E021E9F00E94ED
:10220000BF220E94A922A5E7B3E00E94C7250E9431
:102210009E280E94BF22E0938D03F0938E0360936B
:102220008F03709390030E94CD220E94BA1EAFE3E9
:10223000B3E00E94E81D15C0E0E0E0937503E09371
:102240007603E0937703E0937803E0938D03E093C4
:102250008E03E0938F03E0939003E0933F03E093BA
:102260004003A091AD03B091AE038091AF03909174
:10227000B0030E94B51E0E944127EF930E94D62210
:102280000E944127AF91EA23B9F10E94FB1DE0E0D3
:10229000F0E068EC72E40E94D6260E9497220E9429
:1022A000A3280E94201E0E94D822A0918503B091ED
:1022B00086038091870390918803E0E0F0E064E179
:1022C00072E40E948826DF01CB010E945B1E0E94FF
:1022D000D626A0E0B0E080E291E40E9488260E9429
:1022E000D822E0918503F091860360918703709175
:1022F0008803DE010E944F1E0E944420A091190312
:10230000EDEF0E94A0270E220E944A20E02129F032
:10231000E0911903EF5FE0931903A92D0E944A226F
:10232000A0911903EFEF0E94A0270E220E944A20DD
:10233000E02129F0E894F0F8E0E0E0931903A0919F
:102340001903EEE10E9487270E2E0E944A20E02109
:1023500019F0E1E0E0931C03E0911B03E03019F475
:10236000E0E0E0931C030E94C31E0E94B51E0E9481
:10237000D2270E942121A0911C03E0E00E94A52702
:10238000E02119F0E1E0E0931C03A0911C03AC33C1
:1023900009F41FEFA0910703A13028F0E091070393
:1023A000F0E00E94911F4420C9F4E02FF0E0349641
:1023B0000E94761FAE0FBF1FE12F0E94E122A4E012
:1023C0000E94921DA02F0E94EB22A09135030E9433
:1023D000921DA12F0E94921D0E94F022E1E0E415BF
:1023E00009F057C04424A09113030E94F922E093FE
:1023F0001403F0E0BC96DF01E0911003F0E0AE0FB3
:10240000BF1FE0911103F0E0AE0FBF1FE091120378
:10241000F0E0AE0FBF1FE0911503F0E0AE0FBF1F5D
:10242000EF89F0E0AE0FBF1FE88DF0E0AE0FBF1FE9
:10243000E98DF0E0AE0FBF1FE09116030E94E1228C
:10244000ACE20E94921DA09110030E94921DA091E7
:1024500011030E94921DA09112030E94921DA0914F
:1024600014030E94921DA09115030E94921DAF8932
:102470000E94921DA88D0E94921DA98D0E94921DFE
:10248000A09116030E94EB22A0E00E94EB220E9482
:10249000F022233608F0E0C30E946F222081A0E0E2
:1024A000F799A1E0EA2FE295E07F0E2EA0E0F399E4
:1024B000A1E0EA2FEE0FEE0F0E0EA0E0F499A1E0DE
:1024C000EA2FEE0FA02DAE0FE0E0F599E1E0EA0F64
:1024D000ED8FEAE0EAABEBABECABEDABEEABEFAB29
:1024E000E8AF0E94FF22EAE0ECAFEDAFEEAFEFAF56
:1024F000DE01A05CBF4FEC93E0912403E03021F4B7
:102500000E940423E00DEE8FA0912403A13021F559
:10251000A0E022FCA1E0EA2FEE0FE75F0E2EA0E084
:1025200022FCA1E0EA2FEE0FEE0FE00DEF8FE0911D
:102530002E03E170EE0FE058AE2FE0912E030E94C3
:102540001D23EA0F0E2EA0E0F199A1E0EA2FEE0F75
:10255000EE0FEE0FE00DEE8FA0912403A23099F460
:102560000E9404230E0EA0E022FCA1E0EA2F0E94AC
:1025700023230E0EA0E022FCA1E0EA2FE295E07FEB
:10258000EE0FE00DEE8F0E942823AA34E1E0BE0793
:10259000E0E08E07E0E09E071CF4E1E0E093020338
:1025A0000E942823E9E4F1E060E070E00E9431231A
:1025B000EEE5F1E060E070E00E94CA27E02119F04A
:1025C000E3E0E09302030E942823EDE5F1E060E000
:1025D00070E00E943123E8E6F1E060E070E00E94E4
:1025E000CA27E02119F0E7E0E09302030E942823C4
:1025F000E7E6F1E060E070E00E943123ECE7F1E013
:1026000060E070E00E94CA27E02119F0EFE0E0935B
:1026100002030E942823AC37E1E0BE07E0E08E070A
:10262000E0E09E071CF0EFE1E09302030E94C31E6E
:102630000E9435232CF00E943D230E944323ECABE3
:102640000E943D230E946928EDABA0912D03AA3082
:1026500028F00E94B9220E944E23EAAB0E94542324
:10266000EBAB0E9428230E945C230E944323EEAB25
:102670000E9461230E944323EFAB0E9461230E94CA
:102680006928E8AF2130A1F5EF8DE056EF8F0E9469
:1026900067230E947123A436E0E0BE0720F00E9469
:1026A00071230E9476230E9471230E94C8220E94F7
:1026B00081230E9487230E9471230E948D23DB01C6
:1026C000EC93A0910103AA3010F0E2E0E9AFA091F1
:1026D00001030E949223EAAFA09100030E94B92255
:1026E0000E944E23EBAFA09100030E949223ECAF17
:1026F000223009F052C0EF8DE05CEF8F0E94AC1EDB
:10270000A03AE6E8BE07E1E08E07E0E09E0748F069
:102710000E94AC1EE0EAF6E861E070E00E949823B7
:10272000EBAF0E94AC1E0E94A32348F00E94AC1E97
:10273000E0E1F7E260E070E00E949823ECAF0E94D5
:10274000AC1E0E94AB2338F00E94AC1E0E943920C0
:102750000E949823EDAF0E94AC1E0E94B32338F074
:102760000E94AC1E0E945C230E949823EEAF0E9440
:10277000AC1E0E94352328F00E94BB230E949823A0
:10278000EFAFFE01F1963F96FF93EF930E94BB23BC
:102790000E946528AF91BF91EC93233009F077C078
:1027A000E7E7EAAFE4E7EBAFA0918403AA2392F452
:1027B000E0918103F091820360918303709184031F
:1027C0000E945527E0938103F09382036093830373
:1027D000709384030E94D6220E94201E772312F455
:1027E000E0E4EFAF0E94D6220E94201E0E94C12387
:1027F00010F4E0E4EEAF0E94D6220E94201E0E9458
:10280000CA2310F4E0E4EDAF0E94D6220E94201EFD
:102810000E94D32310F4E0E4ECAF0E94DC230E947A
:10282000A3234CF00E94DC23E0E1F7E260E070E0DB
:102830000E944323ECAF0E94DC230E94AB233CF0B8
:102840000E94DC230E9439200E944323EDAF0E94A6
:10285000DC230E94B3232CF00E94DC230E94E5239A
:10286000EEAF0E94DC230E9435232CF00E94E72368
:102870000E944323EFAFFE01F1963F96FF93EF9343
:102880000E94E7230E946928AF91BF91EC93243006
:1028900009F04BC00E94ED23A0916A03AA2312F411
:1028A0000E94F5230E940024772312F4E0E4EFAFA6
:1028B0000E9400240E94C12310F4E0E4EEAF0E94C5
:1028C00000240E94CA2310F4E0E4EDAF0E9400242B
:1028D0000E94D32310F4E0E4ECAF0E940624A03160
:1028E000E7E2BE071CF00E940B24ECAF0E94062416
:1028F000A83EE3E0BE071CF00E941124EDAF0E9449
:102900000624A436E0E0BE071CF00E941724EEAFB8
:102910000E9406241A972CF00E941D240E94212454
:10292000EFAF0E9424240E9429242530C9F40E947C
:10293000ED23E0E5ECAFA0912C03A43618F00E9443
:102940002E24EEAFA0912C030E94B9220E944E23A8
:102950000E948723A0912C030E949223DB01EC9319
:10296000263069F5EF8DE058EF8FE0E0EAAFE5E063
:10297000EBAFE8E7ECAFA881B981A83EE3E0BE0782
:102980002CF0E8EEF3E00E942124EDAFA881B9819C
:10299000A436E0E0BE072CF0E4E6F0E00E9421243B
:1029A000EEAFA881B981EAE0F0E00E9421240E9404
:1029B0008723A881B981EAE0F0E00E94292427302A
:1029C00009F043C0113010F1ECE0EAAFA12F0E94F2
:1029D000F922E436A0E0FA073CF0A12FB0E0E8ECE1
:1029E000F0E00E942124EBAFA12F0E94F9223A9738
:1029F0003CF0A12FB0E0E4E1F0E00E942124ECAF34
:102A0000A12F0E94F9220E944E231EC0EBE0EAAFE4
:102A10000E943424E436A0E0FA0738F0AB81BC8190
:102A2000E8ECF0E00E943924EBAF0E9434243A979E
:102A300038F0AB81BC81E4E1F0E00E943924ECAFD6
:102A40000E9434240E948123EDAF283009F074C025
:102A50000E946723A0916503B0916603A135EBEF57
:102A6000BE0734F4E1E5FBEFE0936503F093660302
:102A7000A0916503B0916603A03BE4E0BE0734F08B
:102A8000EFEAF4E0E0936503F0936603A091660338
:102A9000AA234AF4E0E4EDAFE0916503F091660308
:102AA0000E94512704C0E0916503F0916603E09312
:102AB0006703F0936803A0916703B0916803ECE3A8
:102AC000F0E00E942528E0934703F09348030E941A
:102AD0003C24ECE30E940228A0916703B0916803B4
:102AE000AE1BBF0BA0934903B0934A0324FE1BC047
:102AF0000E943C241A9710F0E2E0E9AF0E943C24C7
:102B00000E948D23EAAFA0914903B0914A030E942D
:102B1000C8220E948123EBAFA0914903B0914A03E0
:102B20000E948D23ECAFE3E7EEAFE8E3EFAFE4E51F
:102B3000DE01A05CBF4FEC93293009F04BC00E942E
:102B40004124A0916A03AA2312F40E94F5230E9453
:102B50000024772312F4E0E4EFAF0E9400240E94E7
:102B6000C12310F4E0E4EEAF0E9400240E94CA23C7
:102B700010F4E0E4EDAF0E9400240E94D32310F48F
:102B8000E0E4ECAF0E940624A031E7E2BE071CF0AF
:102B90000E940B24ECAF0E940624A83EE3E0BE078F
:102BA0001CF00E941124EDAF0E940624A436E0E040
:102BB000BE071CF00E941724EEAF0E9406241A974D
:102BC0002CF00E941D240E942124EFAF0E94242497
:102BD0000E9429242A30C9F40E944124E0E5ECAF88
:102BE000A0912C03A43618F00E942E24EEAFA091E1
:102BF0002C030E94B9220E944E230E948723A09199
:102C00002C030E949223DB01EC93AC85A130E8F009
:102C1000EF8DEF77EF8FE0912E03E170EE0FAE8D29
:102C2000EA23EE8F0E94FF22E9E7ECAFE0E5EDAF8B
:102C3000EEAFAC850E94B9220E944E230E948723EA
:102C4000AC850E949223DB01EC93F29B05C0EE8DD4
:102C5000EB7FEE8FEF5FEE8F233609F046C451E035
:102C6000503130F40E944B24EAE0EC935F5FF8CFE0
:102C7000AA81EBE50E945224EAE50E948727E02919
:102C800011F0ECE2EA83AA81AD3211F4ECE5EA83BB
:102C9000EA81E03029F4E0911003F0E0EF83F88757
:102CA000AA81A13029F4E0911103F0E0EF83F887C5
:102CB000AA81A23029F4E0911203F0E0EF83F887B3
:102CC000AA81A33029F4E0911303F0E0EF83F887A1
:102CD000AA81A43029F4E0911503F0E0EF83F8878E
:102CE000AA81A53021F4EF89F0E0EF83F887AA816B
:102CF000A63021F4E88DF0E0EF83F887AA81A730B1
:102D000021F4E98DF0E0EF83F887AA81A83029F457
:102D1000E0911603F0E0EF83F887AA81A93019F457
:102D2000E0E0EF83E887AA81AA3019F4E0E0EF83BE
:102D3000E887AA81AB3019F4E0E0EF83E887AA8145
:102D4000AC3021F4E4E2F0E0EF83F887AA81AD3003
:102D500021F40E945B1FEF83F887AA81AE3021F433
:102D6000EB89F0E0EF83F887AA81AF3021F4EC899A
:102D7000F0E0EF83F887AA81A03121F4ED89F0E03B
:102D8000EF83F887AA81A13121F4EF85F0E0EF838A
:102D9000F887AA81A23121F4E889F0E0EF83F8876F
:102DA000AA81A33121F4E989F0E0EF83F887AA81B1
:102DB000A43121F40E94DD1EEF83F887AA81A5319A
:102DC00021F4ED81FE81EF83F887AA81A63129F4F1
:102DD000E0912803F0E0EF83F887AA81A73129F476
:102DE000E0912A03F0E0EF83F887AA81A83129F463
:102DF000E0912903F0E0EF83F887AA81A93121F45B
:102E0000E32FF0E0EF83F887AA81AA3121F40E9432
:102E10009222EF83F887AA81AB3131F4E0915B0312
:102E2000F0915C03EF83F887AA81AC3131F4E0E0E4
:102E300023FCE1E0F0E0EF83F887AA81AD3121F4D3
:102E40000E94B11DEF83F887AA81AE3121F40E9460
:102E5000BD1DEF83F887AA81AF3129F4E091080303
:102E6000F0E0EF83F887AA81A03229F4E0910A0309
:102E7000F0E0EF83F887AA81A13229F4E0910B03F7
:102E8000F0E0EF83F887AA81A23229F4E0910C03E5
:102E9000F0E0EF83F887AA81A33229F4E0910D03D3
:102EA000F0E0EF83F887AA81A43229F4E0910E03C1
:102EB000F0E0EF83F887AA81A53229F4E0911F039F
:102EC000F0E0EF83F887AA81A63229F4E09120038D
:102ED000F0E0EF83F887AA81A73229F4E09121037B
:102EE000F0E0EF83F887AA81A83229F4E091220369
:102EF000F0E0EF83F887AA81A93229F4E091230357
:102F0000F0E0EF83F887AA81AA3229F4E091240344
:102F1000F0E0EF83F887AA81AB3229F4E091250332
:102F2000F0E0EF83F887AA81AC3229F4E091260320
:102F3000F0E0EF83F887AA81AC3529F4E09107032C
:102F4000F0E0EF83F887AA81AD3521F4EC8DF0E055
:102F5000EF83F887AA81AE3521F4E985FA85EF83FE
:102F6000F887AA81AF3521F4EB8DF0E0EF83F88785
:102F7000AA81A03621F4EA8DF0E0EF83F887AA81D8
:102F8000A13629F4E0911B03F0E0EF83F887AA81D2
:102F9000A23629F4E0911803F0E0EF83F887AA81C4
:102FA000A33629F4E0911703F0E0EF83F887AA81B4
:102FB000E0E00E945224E3E00E945724E1E10E94F5
:102FC0005724E2E10E945724E3E10E945724E5E1FF
:102FD0000E945724EBE10E945724EDE10E948727CD
:102FE000E02911F0F69A01C0F698A0E0F699A1E068
:102FF000EA2FE795E0E0E795EF8FE0E0EE8FED8FC9
:10300000E09302030E945C240E942124ECAB0E9406
:103010005C240E945728EDABAF81B885A031E7E270
:10302000BE0728F0E0E1F7E20E943924ECAFAF815F
:10303000B885A83EE3E0BE0728F0E8EEF3E00E9482
:103040003924EDAFAF81B885A436E0E0BE0710F0BB
:103050000E947623AF81B8851A9728F00E946324D6
:103060000E948123EFAFFE01F1963F96BF01AF8131
:10307000B8850E948D23DB01EC93EA81E03061F496
:10308000EDE6EEABE9E7EFABE8E7E8AFEDE6EBAF97
:10309000E4E5ECAFE0E5EDAFAA81E1E10E94522466
:1030A000E2E10E945724E3E10E945724E5E10E94F7
:1030B0005724EDE10E948727E02929F00E9463242C
:1030C0000E948123EFAFE7EAE0937A000E94671F36
:1030D000E7E2E0937A00AA810E94961FAA81EEE0BF
:1030E0000E945724E1E10E948727E02911F0E1E0E6
:1030F0006E2EAA810E949B1FAA81EFE00E94572496
:10310000E2E10E948727E02911F0E2E06E2EAA8119
:10311000E7E00E945224E0E10E9457240E946624C6
:1031200011F0E3E06E2E0E94761FD39708F457C08B
:103130000E94B01F0E94B51FE62D0E94BC1F20F008
:10314000E8ECF0E00E94911FE62D0E94CC1F0E9447
:103150006B24AC91A13008F441C00E9472240E94FB
:10316000EC1F0E94FF284CF40E946B240E947B24D9
:103170000E9447270E94862423C00E948F240E9419
:103180000E20EF930E948F240E941720AF91EA2314
:1031900079F00E946B240E947B240E944C27A0930C
:1031A0007103B0937203809373039093740308C008
:1031B0000E948F240E9420201CF00E9491240EC0A7
:1031C000A0917103B0917203809173039091740385
:1031D0000E9439200E944F280E94911F04C00E9423
:1031E0003E200E949124AA81AD3051F40E9499247E
:1031F0000E94E5230E94A2240E94A924E0E2ED8F10
:10320000AA81A53151F40E9499240E94E5230E94CD
:10321000A2240E94A924E0E6ED8FAA810E94961FB5
:10322000AA81EEE00E945724E1E10E948727E0296D
:10323000A9F00E94B324E4E00E94B72418F00E9491
:10324000BD24EEAB0E94761F1A9728F00E94C1247D
:103250000E948123EFAB0E94C324E8AFAA810E94A1
:103260009B1FAA81EFE00E945724E2E10E9487277A
:10327000E029A9F00E94B324E2E00E94B72418F0EC
:103280000E94BD24EEAB0E94761F1A9728F00E9480
:10329000C1240E948123EFAB0E94C324E8AFAA811E
:1032A000E7E00E945224E0E10E9457240E94662435
:1032B000A9F00E94B324E1E00E94B72418F00E9414
:1032C000BD24EEAB0E94761F1A9728F00E94C124FD
:1032D0000E948123EFAB0E94C324E8AFAA81A431EE
:1032E00099F40E94C524E4E6F0E00E943924EEAB94
:1032F0000E94C5240E94C8220E948123EFAB0E9435
:10330000C5240E948D23E8AFAA81A63121F40E9432
:10331000CA24EBE0EDAFAA81A73121F40E94CA24B0
:10332000E0E4EDAFAA81A83121F40E94CA24ECE0C8
:10333000EDAFAA81A93161F4A0912D030E94B922B9
:103340000E944E23EEAB0E945423EFABE7E7E8AFB9
:10335000AA81AA3199F40E94D124E4E6F0E00E9407
:103360003924EEAB0E94D1240E94C8220E948123FE
:10337000EFAB0E94D1240E948D23E8AFAA81AB312C
:1033800059F4ECE7EAAFE7E7EBAFE8E7ECAF0E9410
:1033900063240E948123EFAFAA81EDE10E945224B1
:1033A000EEE10E948727E029D9F0E3E7EAAFE8E3FE
:1033B000EBAFAA81AD3111F4EEE501C0E8E7ECAF67
:1033C0000E94D6241A9738F00E94D6240E94C82260
:1033D0000E948123EFAB0E94D6240E948D23E8AF88
:1033E000AA810E94961FAA81E6E00E945724E7E086
:1033F0000E948727E02911F0E3E7EAAFAA81EEE017
:103400000E945224EFE00E945724E0E10E948727A7
:10341000E02931F0EDE6EAAFE9E7EBAFE4E5ECAF48
:10342000AA81E1E10E945224E2E10E9457240E9415
:10343000662411F0E8E7EBAFAA81EFE10E949B2739
:103440000E2EE5E20E949627E02139F0EDE6EEAB84
:10345000E8E5EFABEA81EF51E8AFAA81AD3559F568
:10346000E7E7EDAFEEE5EEAFE9E3EFAFFE01F19692
:103470003F96AC8DA083E7EAE0937A000E94711F2B
:103480007E2EE7E2E0937A00E3E6E71538F4A72D15
:10349000B0E0E4E6F0E00E942124EEABE9E0E715BD
:1034A00030F4A72D0E94B9220E944E23EFABA72D26
:1034B0000E949223E8AFAA81AE3521F4EEE5EAAF8F
:1034C000E1E0EBAFAA81AF3521F4EEE5EAAFE2E04F
:1034D000EBAFAA81A03621F4EEE5EAAFE3E0EBAF73
:1034E000AA81A23611F4E0E1ED8F51E0503108F0ED
:1034F00077C00E944B24EC91E03021F40E944B24D1
:10350000EFE3EC930E944B24AC91A63021F40E948F
:103510004B24EDE7EC930E944B24AC91A13021F4B5
:103520000E944B24E6E0EC930E944B24AC91A23025
:1035300021F40E944B24EBE5EC930E944B24AC91C8
:10354000A33021F40E944B24EFE4EC930E944B241F
:10355000AC91A43021F40E944B24E6E6EC930E9447
:103560004B24AC91A53021F40E944B24EDE6EC9362
:103570000E944B24AC91A73021F40E944B24E7E039
:10358000EC930E944B24AC91A83021F40E944B2470
:10359000EFE7EC930E944B24AC91A93021F40E94F8
:1035A0004B24EFE6EC930E944B24AC91AA3021F41B
:1035B0000E944B24E0E0EC930E944B24AC91AB3092
:1035C00021F40E944B24E1E0EC930E944B24AC9147
:1035D000AC3021F40E944B24E8E0EC935F5F86CF8F
:1035E000E0910203E695E6950E94DB24EEA90E9495
:1035F000E124EEA90E94E924EEA90E94F424EEA998
:103600000E94FB24EEA90E940225EEA90E94092532
:10361000EEA90E941025E9A3E0910203E695E69544
:10362000E6950E94DB24EFA90E94E124EFA90E9405
:10363000E924EFA90E94F424E8AD0E94FB24E8AD40
:103640000E940225E8AD0E940925E8AD0E941025E0
:10365000EAA3E0910203E6950E94DB24E8AD0E9414
:10366000E124E8AD0E94E924E8AD0E94F424EFA92A
:103670000E94FB24EFA90E940225EFA90E940925C0
:10368000EFA90E941025EBA3E9AD0E94DB24EAAD6F
:103690000E94E124EAAD0E94E924EAAD0E94F424EC
:1036A000EF8D0E94FB24EF8D0E940225EF8D0E947A
:1036B0000925E0910203E170EA2BECA3EEAD0E9434
:1036C000DB24EEAD0E941625EEAD0E941C25EEAD6A
:1036D0000E9425250E942F25EEAD0E943325EEADD8
:1036E0000E943C25EEADE295E170EA2BEDA3EDAD35
:1036F0000E94DB24EDAD0E941625EDAD0E941C2535
:10370000EDAD0E942525E2950E94FB24EFAD0E94BD
:103710003325EFAD0E943C25EFADE295E170EA2B39
:10372000EEA3EF8D0E944525EDAD0E94E124EDADA5
:103730000E94E924EDAD0E94F424ECAD0E94FB242C
:10374000ECAD0E940225ECAD0E940925ECAD0E9473
:103750001025EFA3EFAD0E94DB24EFAD0E941625EC
:10376000EFAD0E941C25EFAD0E9425250E94492542
:103770000E94FB24ECAD0E943325ECAD0E943C2559
:10378000ECADE295E170EA2BE8A7EBAD0E94DB24FB
:10379000EBAD0E941625EBAD0E941C25EBAD0E94FF
:1037A0002525EE1FE0E0EE1F0E94FB240E944E251F
:1037B0000E9433250E944E250E943C250E944E25E2
:1037C000E295E170EA2BE9A7EE8DE2950E94DB24F9
:1037D000EBAD0E94E124EBAD0E94E924EBAD0E9429
:1037E000F424EAAD0E94FB24EAAD0E940225EAAD72
:1037F0000E940925EAAD0E941025EAA70E944E25E5
:103800000E94DB240E944E250E9416250E944E2510
:103810000E941C250E944E25E695E695E6950E949D
:103820005325EAA9EE1FE0E0EE1F0E94FB24EAA95F
:10383000E295E170EE0FEE0FEA2BAE2FEAA90E949F
:103840003C25EAA9E295EF70E695E170EA2BEBA73B
:10385000EAA9E695E695E6950E94DB24EAA9E695B5
:10386000E6950E945925EAA90E945E25EAA90E94D0
:103870005325EE8D0E942F25EE8D0E941D23EA2BED
:10388000AE2FEE8D0E946625EE8DE695E170EA2B57
:10389000ECA7EE8D0E944525EBA9E2950E945925E3
:1038A000EBA90E94E924EBA90E946B25EBA90E94D9
:1038B0002F25EBA90E941D23EA2BAE2FEBA9E6953D
:1038C0000E946625EBA9E170EA2BEDA7EE8D0E9420
:1038D00049250E94DB24ED8D0E945925ED8D0E9423
:1038E0005E25ED8DE695E6950E945325E091020355
:1038F000E2950E94FB24EE8DEE1FE0E0EE1FE170EA
:10390000EE0FEE0FEA2BAE2FED8DE695E695E695E0
:103910000E946625ED8DE295E170EA2BEEA7ED8D14
:103920000E944525ECA9E2950E945925ECA90E9428
:10393000E924ECA90E946B25EDA90E942F25EDA991
:103940000E941D23EA2BAE2FEDA9E6950E94662565
:10395000EDA9E170EA2BEFA7ED8D0E9449250E94A9
:10396000DB24EDA9E2950E945925EDA90E94E924E6
:10397000EDA90E946B25ECA90E942F25ECA90E94BD
:103980001D23EA2BAE2FECA9E6950E946625ECA933
:10399000E170EA2BE8AB33FE0DC051E0513150F439
:1039A000E52FF0E0DE019096AE0FBF1FEFEFEC9336
:1039B0005F5FF4CF0E946F255D3078F40E9475251B
:1039C000A2E5B8E00E946527E17011F45D9801C09E
:1039D0005D9A0E947C255F5FEFCF0E9484255D3059
:1039E00078F40E947525A0E3B8E00E946527E17095
:1039F00011F45D9801C05D9A0E947C255F5FEFCF56
:103A00000E9484255D3078F40E947525A2E0B8E01C
:103A10000E946527E17011F45D9801C05D9A0E94D3
:103A20007C255F5FEFCF0E9484255D3078F40E9493
:103A30007525A6E0B8E00E946527E17011F45D9855
:103A400001C05D9A0E947C255F5FEFCF0E948425B4
:103A50005A3098F45E9885E28A95F1F7E9E0E51B23
:103A6000A0E4B1E00E946527E17011F45D9801C007
:103A70005D9A0E947C255F5FEBCF41E04131E8F425
:103A800051E05930C0F45E9885E28A95F1F7E42F51
:103A9000F0E0DE019096AE0FBF1FAC91E8E0E51BB1
:103AA0000E945D27E17011F45D9801C05D9A0E944B
:103AB0007C255F5FE6CF4F5FE1CF5D9A85E28A9517
:103AC000F1F7289A8DEC9AE00197F1F70E944420D3
:103AD000A82DEAE00E94A0270E2AAA2DEAE00E9463
:103AE000A0270E2AAD2DEAE00E94A027E02929F0A8
:103AF000E0E0E0934F03E0935003AB2DE4E60E9437
:103B0000A5270E2EA0E0F099A1E00E94602039F0D8
:103B1000A4E6B0E00E948E25F09AE89433F80C9465
:103B20003505FFCFAA93E091C000E072E1F3E88190
:103B3000E093C60021960895A0913903B0913A030D
:103B40000895A0918D03B0918E0380918F03909181
:103B500090030895E0E0F0E061EE75E40E94D6265F
:103B60000895E0914503F09146030895662777276D
:103B70000E94FE250E949E280895E0915103F09135
:103B800052030895A0919503B091960380919703F5
:103B9000909198030895E0E0F0E060E271E4089508
:103BA000A0914503B09146030895E0E0F0E00E9443
:103BB000BC270895A0915103B09152030895E0915C
:103BC000BD03F091BE036091BF037091C0030895DF
:103BD0000E94C525ED93FC930895A091A903B0918F
:103BE000AA038091AB039091AC0308950E948826AC
:103BF000DF01CB01AFCFA091A503B091A6038091C7
:103C0000A7039091A8030895E0915B03F0915C03F2
:103C100060915D0370915E030895A4E6B0E080E0DA
:103C200090E00E94E227DF01CB01E091A503F09133
:103C3000A6036091A7037091A8030E94A32808958A
:103C40000E94A8280E9431260895E0917903F091FE
:103C50007A0360917B0370917C030895A091C50362
:103C6000B091C6038091C7039091C8030895E09373
:103C7000C503F093C6036093C7037093C803089508
:103C80000E94E227DF01CB01E091C503F091C6035A
:103C90006091C7037091C8030E94A328D1CF0E94EE
:103CA000C725ED93FC930895E0E0F0E061EE75E444
:103CB0000E9488260895E091AD03F091AE036091D3
:103CC000AF037091B0030895E091B103F091B20396
:103CD0006091B3037091B4030895A0919103B091E2
:103CE000920380919303909194030895E09391033C
:103CF000F093920360939303709394030895A091BB
:103D00009903B0919A0380919B0390919C0308952D
:103D1000E0919103F0919203609193037091940369
:103D20000895A091A103B091A2038091A303909163
:103D3000A4030895E0915703F0915803609159034B
:103D400070915A030895E0935703F09358036093DA
:103D5000590370935A030895A0915703B0915803E3
:103D60008091590390915A030895E0E0F0E060E0FB
:103D700070E0089510DF0E9488260895E0E00E9418
:103D8000A5270E2E0895A0917503B091760380911A
:103D900077039091780308950E22A0911C03ECE321
:103DA0000E94A0270895A0914F03B0915003089559
:103DB000A0914D03B0914E03F8CEE0914D03F091E8
:103DC0004E030895E7EAE0937A00A4E00E943303EB
:103DD000EF2FF0E09E2EE7E2E0937A00E7EAE0932F
:103DE0007A000895A3E00E943303EF2FF0E08E2EB7
:103DF000E7E2E0937A00E7EAE0937A000895A1E031
:103E00000E943303EF2FF0E0AE2EE7E2E0937A005A
:103E10000895E0E0F0E00E94D1280895EBE0E093FF
:103E2000CE03E8EBE093CF030895E8ECF0E0E093F5
:103E30006103F09362030895E0EDF7E0E09363031C
:103E4000F09364030895E0933D03F0933E030895D7
:103E50000E947D270E94FE250E949E280895E093DF
:103E60004303F09344030895E0935B03F0935C03F2
:103E700060935D0370935E030895E0934D03F093A8
:103E80004E030895E7EAE0937A00A0E00E9433032E
:103E9000EF2FF0E008950E9433030E9472270E94E2
:103EA0006E270895E0937903F0937A0360937B0380
:103EB00070937C030895E0913D03F0913E030895D3
:103EC000E7E2E0937A00E7EAE0937A000895A7E05A
:103ED0000E943303EF2FF0E0E0933503F0933603B5
:103EE00008950E943303EF2FF0E00895A091350369
:103EF000B09136030895FADFEAEFF0E00895F6DFB7
:103F0000EEE1F0E00E94B62708950E2EA52DE1E027
:103F10000E94A5270E22AC85E5E00E94A027E021A3
:103F20000895E0933503F09336030895E5E00E9489
:103F300087270E2E0895E6E00E9487270E2E08950B
:103F4000AD2DEAE00E94A0270E2E0895A0E0F3FC1C
:103F5000A1E0E0E00E9487270E22A22FE3E6089569
:103F6000E0913503F09136030895F297ADE7B0E0A4
:103F70000E94DA270F010895F0E0DE015296AE0F9D
:103F8000BF1FEC91F0E0D0010E941228CADFAEDF23
:103F9000A93CE0E0BE070895F0E0DE015696AE0FC2
:103FA000BF1FEC91F0E0A2DF0E94DA27DF01E4E618
:103FB000F0E00E941228B5CFE02FF0E0DE011E965F
:103FC000AE0FBF1F0895A0916D03B0916E03809155
:103FD0006F03909170030895E8EEF3E060E070E005
:103FE0000E944F28DF01CB01BBDF662777270895AA
:103FF000EC91F0E00E947D27A8E0BCE481E090E035
:104000000E944F28E0CFE0936D03F0936E0360931E
:104010006F03709370030895D6DFDECF0E944C27A4
:10402000E5E0F0E060E070E00E94D22708950E9491
:104030004C27E4E1F0E060E070E00E94CA270895B8
:104040000E944C27A431E0E0BE07E0E08E07E0E0EC
:104050009E070895E0917503F091760360917703D0
:1040600070917803A0E5B4E180E090E00E940D2813
:10407000CACFE8EEF3E060E070E00895E0E0E0939E
:104080003503E09336030895A92DEAE00E94A027A6
:104090000E2E0895A22FE3E60E94A0270895A0E027
:1040A000F0FCA1E0E0E00E9487270895A0912B0397
:1040B00065CEE0912A0367DEFF27662777270895FC
:1040C000E0E00E948727E0210895ED81FE81A09124
:1040D0007903B0917A0380917B0390917C036627EA
:1040E00077270E94CA270E2EEAE0F0E060E070E039
:1040F0000E94D2270895E0936103F093620308952C
:10410000A4DDAD81BE81882799270E944C270895A0
:10411000A630E0E0BE07E0E08E07E0E09E070895ED
:10412000A0916103B09162030895E0916103F09161
:1041300062030895ED81FE81A0917903B0917A0325
:1041400080917B0390917C03662777270895E32F66
:10415000A091B903B091BA038091BB039091BC03C5
:10416000FF27662777270E94FE250895BFDEEAE035
:104170000E9402280895E32FF0E0A091B903B091C6
:10418000BA038091BB039091BC030E947D270E94DB
:10419000FE2556CD662777270E94FE250E94882699
:1041A0000895A0916303B091640308950E9482274B
:1041B0000E94A52845CDA32FBB27E091B903F0911C
:1041C000BA036091BB037091BC03F0CFE09163032D
:1041D000F09164030895EAE0F0E00E942528A1CE62
:1041E000E0911203D0DDFF27662777270895E0933B
:1041F0006B03F0936C030895E0911203F0E0C3DDCC
:104200000E947D270E944C2708950E940828A091B3
:104210006B03B0916C030895E0916B03F0916C0314
:104220000895A0911203BB27E0917503F0917603E6
:1042300060917703709178030E9482270E944C2737
:1042400008950E2EA0911C03ECE30E94A0270E22DD
:104250000895E0911103A0E0B0E00E94D928A1E008
:10426000B0E00E948E25E0911203A1E0B0E00E9430
:10427000D928A1E0B0E00E948E25E0911303A2E0CE
:10428000B0E00E94D928A1E0B0E00E948E25E09124
:104290001503A3E0B0E00E94D928A1E0B0E00E949D
:1042A0008E25EF89A4E0B0E00E94D928A1E0B0E01B
:1042B0000E948E25E88DA5E0B0E00E94D928A1E0FB
:1042C000B0E00E948E25E98DA6E0B0E00E94D928DA
:1042D000A1E0B0E00E948E25E0911603A7E0B0E0D7
:1042E0000E94D928A1E0B0E00E948E25E09117033A
:1042F000A8E0B0E008950E94D928A1E0B0E00C94B5
:104300008E25E0911803A9E0B0E0F5CFE0911B0302
:10431000AAE0B0E0F0CFCFDDA6E2B0E00E94D12865
:10432000A1E0B0E00E948E25EB89A4E1B0E0E3CFEC
:10433000ED81FE81AAE2B0E00E94D128A1E0B0E0C8
:104340000E948E25E0912803AEE0B0E0D4CFE0914A
:104350002A03AFE0B0E0CFCFE0912903A0E1B0E0C5
:10436000CACFE985FA85ACE2B0E00E94D128A1E08D
:10437000B0E00E948E25EB8DA2E1B0E0BCCFE091D1
:10438000A503F091A6036091A7037091A803AEE284
:10439000B0E00E94C7250E94D128A1E0B0E00E94B1
:1043A0008E25E0914303F0914403A0E3B0E00E9426
:1043B000D128A1E0B0E00E948E25E0915B03F0914E
:1043C0005C03A4E3B0E00E94D128A1E0B0E00E9429
:1043D0008E25E0E023FCE1E0A7E1B0E08CCFEDDC4E
:1043E000A2E3B0E00E94D128A1E0B0E00E948E25B7
:1043F000E0910803A8E1B0E07ECFE0910A03A9E1D3
:10440000B0E079CFE0910B03AAE1B0E074CFE09186
:104410000C03ABE1B0E06FCFE0910D03ACE1B0E095
:104420006ACFE0910E03ADE1B0E065CFA6E3B0E066
:104430000E94C7250E94D128A1E0B0E00E948E25ED
:10444000E0911F03AEE1B0E056CFE0912003AFE171
:10445000B0E051CFE0912103A0E2B0E04CCFE09179
:104460002203A1E2B0E047CFE0912303A2E2B0E053
:1044700042CFE0912403A3E2B0E03DCFE0912503D9
:10448000A4E2B0E038CFE0912603A5E2B0E00E94BC
:10449000D9280895EAE00E94A5270E2E0895AA2D96
:1044A000EAE00E94A0270E2EA0E027FCA1E0E0E0B9
:1044B0000E9487270E220895A0E0F2FCA1E0E0E030
:1044C0000E9487270E220895A82DEAE00E94A027C7
:1044D0000E2E0895E0E00E9487270E220895E091B5
:1044E0000F03F0E0E65FFC4F08950E22A22FE3E6F3
:1044F0000E948727E0210895A22FE3E60E948727E4
:10450000E0210895E0913203EF5FE0933203E09100
:104510003103A0913203EA170895A0914303B091AB
:1045200044030895E0914303F09144030895A0915A
:104530005B03B0915C0380915D0390915E030895ED
:10454000E091B903F091BA036091BB037091BC0391
:104550000895A0E0B0E080E09FE30E94382608952F
:10456000E093A903F093AA036093AB037093AC03A9
:104570000895B0E0EAE0F0E00E9425280895E09177
:104580008903F0918A0360918B0370918C030895E5
:10459000EAE0F0E00E9412280895A0918903B0910A
:1045A0008A0380918B0390918C0308952DDB35CB8A
:1045B000E0938503F09386036093870370938803E9
:1045C0000895F0E0EA0FFB1FE0934103F0934203EC
:1045D000AEE30C94921D0E94921DA0E00C94921DDB
:1045E000E0914203AE2F0E94921DA09141030C94D2
:1045F000921DB0E0E2E0F0E00E9425280895EAE094
:10460000E9AFEAAFEBAF0895E9E0EF8FE0912E0359
:10461000E170EE0FE058AE2FE0912E03E695E6959F
:10462000E170EE0FEE0FEA0F0E2EA0E0F199A1E07F
:10463000EA2FEE0FEE0FEE0F0895E695E695E17086
:10464000EE0FEE0F0895E295E07FEE0FEE0F089566
:10465000A0917D03B0917E0380917F0390918003B0
:1046600008950E94D2270E2EF3CFAA30E0E0BE07B5
:10467000E0E08E07E0E09E07089585DBEAE0F0E0E9
:1046800060E070E008950E944F28DF01CB01EAE06E
:10469000F0E060E070E00E9469280895DF01EAE040
:1046A000F0E00E9457280895A0912D03BB27EAE06F
:1046B000F0E00E9457280895E4E6F0E060E070E042
:1046C0000895C6DFEAE0F0E060E070E00895A0E061
:1046D00020FCA1E0EA2FE295E07FAE8DEA0FEE8F9D
:1046E0000895A0913B03B0913C030895E4E6F0E007
:1046F0000E941228DF01EAE0F0E00E945428EEAFA9
:104700000895DF01EAE0F0E00E9454280895EFAF39
:10471000FE01F1963F96BF010895EAE0F0E00E94A5
:1047200054280895BB27EAE0F0E00E945728089536
:104730000E942A28DF01CB01EAE0F0E060E070E0AF
:104740000E9465280895A031E7E2BE07E0E08E07E9
:10475000E0E09E070895A83EE3E0BE07E0E08E0794
:10476000E0E09E070895A436E0E0BE07E0E08E0793
:10477000E0E09E070895F0DAEAE0F0E060E070E043
:104780000895DF01CB01E0E0F0E060E171EC0E9410
:104790001B270895DF01CB01E0E0F0E066EC72EC4E
:1047A0000E941B270895DF01CB01E0E0F0EC69E7F0
:1047B00074EC0E941B270895A0918103B09182039D
:1047C0008091830390918403089576DF5CCFF4DFBA
:1047D000EAE0F0E060E070E00895EF8DE058EF8FE0
:1047E000EEE3EAAFE4E7EBAF0895E0916903F091FF
:1047F0006A030E945127E0936903F0936A030895C6
:1048000003DAA4E6B0E080E090E03ACAA091690340
:10481000B0916A030895FADFE0E1F7E20E942528EB
:104820003DCFF4DFE8EEF3E00E94252837CFEEDF3E
:10483000E4E6F0E00E94252831CFE8DFEAE0F0E08E
:1048400008950E9425282ACFFE01F1963F96BF01C8
:10485000F4CF0E945728DB01EC930895A0912C031C
:10486000B0E0E4E6F0E0EDCFEB81FC81F695E79572
:1048700008950E94122845CFA0914703B0914803A4
:104880000895EF8DE058EF8FE2E0E9AFEEE3EAAF95
:10489000E4E7EBAF0895E52FF0E0DE01D196AE0F2F
:1048A000BF1F08950E9487270E2EAA8108950E9497
:1048B00087270E2AAA810895AA81B0E0A7FDBFEF3D
:1048C000EAE0F0E00895AF81B88562CEE3E10E94AE
:1048D0008727E0290895E62DF0E0DE011E96AE0F51
:1048E000BF1F0895A0917103B0917203809173036B
:1048F000909174030895EC91F0E00E947D27A8E068
:10490000BCE481E090E00E944F28ECCFE09371037B
:10491000F093720360937303709374030895E2DF5E
:104920005BCBE985FA852FDA662777270E940D2869
:10493000EDCFA0917903B0917A0380917B039091A0
:104940007C030895EEABF5DFEAE0F0E060E070E0B4
:104950009ACEEFABEEDFEAE0F0E060E070E00E94BC
:104960006928E8AF0895FCDAF695E795DACAED8F85
:10497000BDDAA436E0E0BE070895B8DAE4E6F0E078
:1049800078CFB4DA05CEB2DAC8CEA0915503B09193
:1049900056030895E9E3EAAFE0E5EBAFEEE3ECAFF1
:1049A0000895A0913F03B09140030895A0914B0357
:1049B000B0914C030895E170E795E0E0E795AE2FE4
:1049C0000895E295EF70E695E1703DDEEA2BAE2F9B
:1049D0000895E295EF70E695E695E170E295E07F47
:1049E000EE0FEA2BAE2F0895E295E170E295E07F9D
:1049F000EA2BAE2F0895E170EE0FEE0FEE0FEA2BCB
:104A0000AE2F0895E695E170EE0FEE0FEA2BAE2F74
:104A10000895E695E695E170EE0FEA2BAE2F089526
:104A2000E695E695E695E170EA2B0895E695E17046
:104A30000ADEEA2BAE2F0895E695E695E170E29541
:104A4000E07FEE0FEA2BAE2F0895E695E695E6950A
:104A5000E170E295E07FEA2BAE2FEF8D0895E695A9
:104A6000E695E695C8CFE295EF70E695E170EE0F1A
:104A7000EE0FEA2BAE2F0895E295EF70E695E695DE
:104A8000E170EE0FEA2BAE2F0895E295EF70E695F8
:104A900092CFE295EF70E695E6950895FE01E05C11
:104AA000FF4FE0810895E170E295E07FEA2BAE2FA1
:104AB0000895E170C8DDEA2BAE2F0895E695E17008
:104AC000E295E07FEE0FEA2BAE2F0895E170EE0F36
:104AD000EA2BAE2F0895E295EF70E695E4CF289883
:104AE00085E28A95F1F751E008955E9885E28A950E
:104AF000F1F7ECE0E51B089585E28A95F1F75E9AFF
:104B000085E28A95F1F708955D9A85E28A95F1F735
:104B1000289A84E191E00197F1F7E1CF109639F0FE
:104B20008DEC9AE00197F1F7A8951197C9F70895D0
:104B3000552342F4503811F4E0FF04C03196691F48
:104B4000791F6BF050E8572711F45F93CFC05F3F98
:104B500031F0660F000C57956795752F08955F9398
:104B600000200AF0CFC0C8C050E8192E1522880FC7
:104B7000991F9527550F879550E8072E0522660F38
:104B8000771F7527550F67950895689401C0E894BD
:104B90005F93F2DF703818F07F3F08F4A7C056E14A
:104BA000571BAAF4519558300EF4593030F0EFEFFE
:104BB000FFEF6FEF7FE777F91AC077275523B9F03A
:104BC000EE0FFF1F661F771F5A95D1F710C077278A
:104BD000583028F0EF2FF62F672F5850F9CF552374
:104BE00031F076956795F795E7955A95D1F70020BE
:104BF0000AF45BD15F910895689401C0E8943097FE
:104C000060407040B1F0002426F0772312F4009445
:104C10004CD1172E7EE1112032F07A95EE0FFF1F56
:104C2000661F111CF9CFEF2FF62F612D5F938ADFDE
:104C30005F9108954F93AF01FD01DA01AB01BC0113
:104C4000CA01402D012C142E4F910895EA0FFB1F2D
:104C5000681F0895E095F0956095EF5FFF4F6F4FE7
:104C600008955F9381DF903871F150E8152604C0F4
:104C70005F937ADF903839F1703821F1572F591B43
:104C80002BF112F4D7DFFACF583118F0AA27BB273F
:104C90008827583028F0AB2FB82F88275850F9CFE5
:104CA000552329F08695B795A7955A95D9F7502D94
:104CB000512572F0CBDF38F46795F795E79573953A
:104CC00013F420C0B7DF3EDF5F910895D8F7FBCF24
:104CD000EA1BFB0B680B51F010F40094BBDF66235A
:104CE00092F3EE0FFF1F661F7A95CBF7EE27FF2793
:104CF000662777275F910895EFEFFFEF6FE77FEF6C
:104D00005F910895EFEFFFEF6FE77FE75F91089501
:104D10005F932ADF703851F3903841F301240894EF
:104D2000791F23F41CF300203AF3ECCF0F921F936A
:104D30002F933F934F93112722279927689FA00114
:104D40008F9F302D410D591F6B9F300D411D591FF5
:104D50008E9F27D0BF9F25D06A9F23D0BE9F1DD096
:104D6000AF9F1BD0AE9F110D291F391F491F591F1F
:104D7000E32FF42F652F522F4F913F912F911F91C9
:104D80000F9066232AF0550FEE1FFF1F661F02C00B
:104D900073954BF2CDDE5F910895100D211D391FE3
:104DA00002C0200D311D491F591F08955F93DCDE9D
:104DB000703821F411200AF49FCFA4CF903809F461
:104DC00095CF01240894970B1BF4D4F30020F3CF64
:104DD000792F1F932F933F934F931124112722274D
:104DE00033274427552790E2AE17BF0786074107B0
:104DF00030F0AE1BBF0B860B410B089401C08894AA
:104E0000551F221F331F111CAA1FBB1F881F441FC1
:104E10009A9551F7F901612D4F913F912F911F9173
:104E2000662332F0550FEE1FFF1F661F7A9543F27F
:104E30007FDE5F91089599239AF0772342F09717C8
:104E400048F029F4AE17BF07860720F031F0989498
:104E500088940895989408940895189488940895CF
:104E60007723C2F7971798F3A9F7EA17FB076807A4
:104E700088F399F3ECCFDFDFE1E009F008F0EE27EB
:104E80000895D9DFE1E009F008F4EE270895EA0F6C
:104E9000FB1F681F791F0895AE1BBF0B860B970B76
:104EA0000895F195E195F0400895F095609570951D
:104EB000E195FF4F6F4F7F4F0895EE230E2EEA2F9F
:104EC00019F0E6950A94E9F70895EE230E2EFD01F8
:104ED00021F0F695E7950A94E1F70895F695E795A0
:104EE000F695E795F695E795F695E7950895FE2FE3
:104EF000FF0FFF0B6F2F7F2F08956F2F660F660B2D
:104F0000762F08958B2F880F880B982F0895EA1716
:104F1000E1E009F0EE270895EA17E1E009F4EE2751
:104F20000895AE17E1E00CF4EE270895AE17E1E026
:104F30000CF0EE270895EA17E1E00CF0EE27089553
:104F4000AE17E1E008F0EE270895EA17E1E008F077
:104F5000EE270895EA17FB07E1E009F0EE27089530
:104F6000AE17BF07E1E008F4EE270895AE17BF07BC
:104F7000E1E008F0EE270895EA17FB07E1E008F00A
:104F8000EE270895EA17FB0768077907E1E009F0C3
:104F9000EE270895AE17BF0786079707E1E00CF0EC
:104FA000EE270895EA17FB0768077907E1E00CF0A0
:104FB000EE270895FA9FF02DEB9FF00DEA9FE02D6C
:104FC000F10D08957A9F702D6B9F700DF89F700DF5
:104FD000E99F700D6A9F602D710DFB9F600D711D23
:104FE000E89F600D711D8827FA9FF02D610D781FD5
:104FF000EB9FF00D611D781FEA9FE02DF10D681FFA
:10500000781F08956E2F6A9FF0016B9FF00D089531
:1050100074D0D0DF0EF445DF08957DD0D3DF0EF4D9
:1050200044DF08950024112490E1AA0FBB1F001C47
:10503000111C0E1A1F0A18F40E0E1F1E01C0A160CB
:105040009A9599F7FD01D001089557D0EBDF0EF442
:1050500028DF08953F934F935F9300241124442742
:10506000552730E2AA0FBB1F881F991F001C111C77
:10507000441F551F0E1A1F0A460B570B28F40E0E1D
:105080001F1E461F571F01C0A1603A9559F7FD0129
:10509000BC01D001CA015F914F913F9108953BD06F
:1050A000D9DF0EF402DF0895BDDFFD010895E89415
:1050B000B7FF04C0A095B09511966894F7FDF1DE96
:1050C000B1DFFD010EF4EDDE0895C4DFFD01BC018A
:1050D0000895E89497FF09C0A095B09580959095A4
:1050E000AF5FBF4F8F4F9F4F689477FDDEDEB2DF1B
:1050F000FD01BC010EF4D9DE0895E894F7FF02C06B
:10510000D0DE6894B7FF06C0A095B095119600F860
:10511000039400FA0895E89477FF02C0C6DE68940D
:1051200097FF0BC00024A095B0958095909511969F
:10513000801D901D00F8039400FA0895ED93FD93EF
:105140006D937C930895689401C0E89401D057DD75
:10515000182E862F612D192E972F712D1B2EBF2FE4
:10516000F12D1A2EAE2FE12D0895129602D0BF0117
:105170001297119602D0FE2F1197F999FECFFF9347
:10518000FFB7F894A1BDB2BDF89AE0B5FFBFFF919B
:10519000089507D012960F01FB0103D0F00112977A
:1051A000089507D01196EF93EF2F03D0EF91119749
:1051B0000895F99B02C0A895FCCF9FB7F894A1BDB4
:1051C000B2BDF89A80B5E81719F0E0BDFA9AF99ADD
:1051D0009FBF089500240E160F06060607060895C1
:1051E00000240A160B06089500240A160B0608066A
:1051F00009060895EA17FB07680779070895AE17AF
:10520000BF07860797070895E894EE2309F068948E
:105210000895AC0FBD1F05900D928A95E1F7089592
:00000001FF
